:0200000480007A
:100000006F00C004732F2034930F8000630AFF0336
:10001000930F90006306FF03930FB0006302FF038A
:10002000170F0080130F0FFE63040F0067000F000F
:10003000732F203463540F006F00400093E19153FD
:10004000171F000023203FFC6FF09FFF732540F136
:1000500063100500970200009382020173905230F2
:10006000735000189702000093820202739052307E
:10007000B70200809382F2FF7390023B9302F0017B
:100080007390023A9702000093828201739052307B
:100090007350203073503030735040309301000063
:1000A00097020000938242F67390523013051000BD
:1000B0001315F501634C05000F00F00F93011000BC
:1000C0009308D0051305000073000000970200801C
:1000D000938242F3638E020073905210B7B2000015
:1000E000938292107390223073232030E39862F44D
:1000F00073500030970200009382420173901234D3
:10010000732540F173002030930010001397000016
:10011000930E100093012000631AD727930010005C
:1001200013971000930E2000930130006310D7271F
:100130009300100013977000930E00089301400085
:100140006316D725930010001397E000B74E000008
:1001500093015000631CD723930010001397F00104
:10016000B70E0080930160006312D7239300F0FF65
:1001700013970000930EF0FF930170006318D721CE
:100180009300F0FF13971000930EE0FF930180009F
:10019000631ED71F9300F0FF13977000930E00F8B3
:1001A000930190006314D71F9300F0FF1397E000B2
:1001B000B7CEFFFF9301A000631AD71D9300F0FF95
:1001C0001397F001B70E00809301B0006310D71DA4
:1001D000B72021219380101213970000B72E212100
:1001E000938E1E129301C0006312D71BB7202121EA
:1001F0009380101213971000B74E4242938E2E2414
:100200009301D0006314D719B720212193801012D5
:1002100013977000B79E9090938E0E089301E000A4
:100220006316D717B7202121938010121397E0008F
:10023000B74E48489301F000631AD715B720212123
:10024000938010121397F001B70E00809301000104
:10025000631ED7139300100093907000930E000854
:10026000930110016394D013130200009300100057
:10027000139770001303070013021200930220006B
:10028000E31652FE930E0008930120016310D31170
:1002900013020000930010001397E0001300000009
:1002A000130307001302120093022000E31452FE0E
:1002B000B74E000093013001631AD30D1302000002
:1002C000930010001397F0011300000013000000CA
:1002D000130307001302120093022000E31252FEE0
:1002E000B70E0080930140016312D30B130200008C
:1002F0009300100013977000130212009302200065
:10030000E31852FE930E0008930150016310D709C1
:100310001302000093001000130000001397E00088
:100320001302120093022000E31652FEB74E0000A3
:1003300093016001631CD7051302000093001000B5
:1003400013000000130000001397F00113021200C5
:1003500093022000E31452FEB70E00809301700157
:100360006316D7039310F001930E000093018001F0
:10037000639ED0019300100213904001930E000081
:10038000930190016314D001631030020F00F00F4D
:10039000638001009391110093E111009308D0054F
:1003A00013850100730000000F00F00F930110008F
:1003B0009308D0051305000073000000731000C0FF
:0403C0000000000039
:1010000000000000000000000000000000000000E0
:1010100000000000000000000000000000000000D0
:1010200000000000000000000000000000000000C0
:1010300000000000000000000000000000000000B0
:081040000000000000000000A8
:040000058000000077
:00000001FF
